:020000040000FA
:040000006A303A2800
:08000800A000030EA100831209
:1000100005191128831601178312B2308100B0012F
:100020002C2883160113831203140B190310A80D37
:10003000A90DAA0DAB0DAC0DAC16FF302C02031DA3
:100040002C28FA302B02031D2C2831152A08AF006A
:100050002908AE002808AD008B100B11210E83007B
:06006000A00E200E0900B5
:0C007400203084008001840A80300402E7
:10008000031C3C284C2283160C3085058701831203
:10009000850187010730990000309A0010308316DF
:1000A0008E008312603083168F0083120030831617
:1000B00091009F008312C830831681008312313073
:1000C0009000003083168C00831210308B00BC1B14
:1000D0006F2885196F286400851D6B287D233C1CC3
:1000E0007228072381018E018F010B118B100B10D9
:1000F0008C018B178A20311996202922B30B88286E
:10010000031085190314B90DF03039020319B82111
:100110001C237A2864003210B00A301F9528AC01E5
:10012000AB01AA01A901A801B001080031110130F9
:10013000B7008B132030370783169B001C141A0856
:100140008312A4001030370783169B001C141A0872
:100150008312A300A6000230A606003037078316DC
:100160009B001C141A088312A200A7000130A706E6
:100170008B17321CC12822090339A200A309A40944
:10018000A50924082F02031DB22923082E02031DEE
:100190003B2922082D02031DB22901303702031D1D
:1001A000D8283C19D7283D18D8283D143E14712270
:1001B00002303702031DE3283C19E228BD18E3286A
:1001C000BD143E14782203303702031DEE283C197B
:1001D000ED283D19EE283D153E147F2204303702EC
:1001E000031DF9283C19F828BD19F928BD153E143E
:1001F000862205303702031D04293C1903293D1AC4
:1002000004293D163E148D2206303702031D0F29A6
:100210003C190E29BD1A0F29BD163E149422073031
:100220003702031D1A293C1919293D1B1A293D17AC
:100230003E149B2208303702031D25293C1924292E
:10024000BD1B2529BD173E14A22209303702031D0C
:1002500030293C192F294218302942143E14A92272
:100260000A303702031D3B293C193A29C2183B29A1
:10027000C2143E14B02226082E02031DB2292708FC
:100280002D02031DB22901303702031D4E293C19EE
:100290004D293D1C4E293D103E14B7220230370235
:1002A000031D59293C195829BD1C5929BD103E145C
:1002B000BB2203303702031D64293C1963293D1D0D
:1002C00064293D113E14BF2204303702031D6F29FB
:1002D0003C196E29BD1D6F29BD113E14C322053086
:1002E0003702031D7A293C1979293D1E7A293D12CE
:1002F0003E14C72206303702031D85293C19842984
:10030000BD1E8529BD123E14CB2207303702031DC6
:1003100090293C198F293D1F90293D133E14CF226F
:1003200008303702031D9B293C199A29BD1F9B29C0
:10033000BD133E14D32209303702031DA6293C19F0
:10034000A529421CA62942103E14D7220A303702A2
:10035000031DB1293C19B029C21CB129C2103E1499
:10036000DB22B229B70A0B3037020318080099289C
:100370000130B600B300B400B500B70085018701B5
:10038000B1138A20B30BF829031085190314B90D92
:10039000F030390203191F2AB40BF8290130370253
:1003A0000319DF22023037020319E3220330370238
:1003B0000319E722043037020319EB220530370214
:1003C0000319EF22063037020319F32207303702F0
:1003D0000319F722083037020319FB2209303702CC
:1003E0000319FF220A303702031903239630B400A1
:1003F000311DC1293111321C022A2D090339AD00EA
:10040000AE09AF092F1CC1298E018F010C1CC12917
:100410000C102E1EC1298B1320303707BB002F086C
:10042000BA00372210303707BB002E08BA00372237
:1004300000303707BB002D08BA0037228B17850123
:100440008701B70AB6010B303702031CC129072305
:1004500008003E1C08003E101030BB003D08BA00EA
:1004600037223030BB004208BA00372208008B1315
:100470003A0883161C159A0083123B0883169B00CA
:1004800055309D00AA309D009C1464009C18452A9C
:100490001C1183128B170800831600309B001C145C
:1004A0001A088312BC00831610309B001C141A0813
:1004B00083123C18BD00831630309B001C141A08B0
:1004C00083123C18C200831620309B001C141A08AB
:1004D0008312C1000130C11BC100C1080319C10052
:1004E0000800051640084107D0000F08D100080099
:1004F000851640084107D2000F08D30008000514F4
:1005000040084107D4000F08D500080085144008B2
:100510004107D6000F08D70008008714400841079C
:10052000D8000F08D9000800071540084107DA0075
:100530000F08DB000800071440084107DC000F0823
:10054000DD000800871640084107DE000F08DF00C5
:100550000800071640084107CC000F08CD0008002E
:10056000871540084107CE000F08CF00080005128C
:100570008E018F01080085128E018F010800051081
:100580008E018F01080085108E018F0108008710F1
:100590008E018F01080007118E018F0108000710DE
:1005A0008E018F01080087128E018F01080007124B
:1005B0008E018F01080087118E018F010800050848
:1005C000103A850008000508203A85000800050853
:1005D000013A850008000508023A8500080007086E
:1005E000023A870008000708043A87000800070855
:1005F000013A870008000708203A8700080007082A
:10060000103A870008000708083A870008003D18DC
:100610000516BD1885163D190514BD1985143D1A1A
:100620008714BD1A07153D1B0714BD1B87164218FA
:100630000716C218871508003C1D08005008400224
:10064000031D272B51080F02031C272B05125208EC
:100650004002031D302B53080F02031C302B851260
:1006600054084002031D392B55080F02031C392B77
:10067000051056084002031D422B57080F02031CA9
:10068000422B851058084002031D4B2B59080F02BE
:10069000031C4B2B87105A084002031D542B5B0888
:1006A0000F02031C542B07115C084002031D5D2B35
:1006B0005D080F02031C5D2B07105E084002031D3E
:1006C000662B5F080F02031C662B87124C08400242
:1006D000031D6F2B4D080F02031C6F2B07124E08D2
:1006E0004002031D782B4F080F02031C782B871143
:1006F0000C1C08000C10C00A0800B601B301B401BC
:100700003C1C852BBC01BC148C2BBC1C8A2BBC0153
:100710003C158C2BBC013C143C08B6006400902BAB
:10072000912B922B932B942BB41B0516B41F0512FF
:10073000B30B8E2BB40B8E2B0310B60CB608031D17
:0E0740008E2B0030BB003C08BA0037220800A8
:084000000900030006000600A0
:02400E00CC33B1
:10420000010078007A007C007E007B0079007F004E
:104210007D007A0078007E007C00FF00FF00FF0038
:104220000000F200F600FA00FE00F200F600FA00CC
:10423000FE00F200F600FA00FE00FF00FF00FF00A3
:10424000010005000500050005000900090009003E
:1042500009000D000D000D000D00FF00FF00FF0024
:104260000000FF00FF00FF00FF00FF00FF00FF0055
:10427000FF00FF00FF00FF00FF00FF00FF00FF0046
:10428000FF00FF00FF00FF00FF00FF00FF00FF0036
:10429000FF00FF00FF00FF00FF00FF00FF00FF0026
:1042A000FF00FF00FF00FF00FF00FF00FF00FF0016
:1042B000FF00FF00FF00FF00FF00FF00FF00FF0006
:1042C000FF00FF00FF00FF00FF00FF00FF00FF00F6
:1042D000FF00FF00FF00FF00FF00FF00FF00FF00E6
:1042E000FF00FF00FF00FF00FF00FF00FF00FF00D6
:1042F000FF00FF00FF00FF00FF00FF00FF00DD00E8
:00000001FF
